:100000000C9446000C9465000C9465000C946500FB
:100010000C9465000C9465000C9465000C946500CC
:100020000C9465000C946E000C9465000C946500B3
:100030000C9465000C9465000C9465000C946500AC
:100040000C9465000C9465000C9465000C9465009C
:100050000C9465000C9465000C9465000C9465008C
:100060000C9465000C9465000C9465000C9465007C
:100070000C9465000C9465000C9465000C9465006C
:100080000C9465000C94FA020C94650011241FBEB8
:10009000CFEFD0E1DEBFCDBF11E0A0E0B1E0E4E6FC
:1000A000F8E000E00BBF02C007900D92A030B1074E
:1000B000D9F711E0A0E0B1E001C01D92AF3EB10759
:1000C000E1F70E94BB000C9430040C9400008BE01C
:1000D00085BD89EF83BD80E887BF08951F920F9289
:1000E0000FB60F9211248F939F93AF93BF9380917C
:1000F000010190910201A0910301B09104010196C8
:10010000A11DB11D8093010190930201A0930301F1
:10011000B0930401809100018F5F809300018A30C9
:1001200059F4109200018091050190910601019609
:100130009093060180930501BF91AF919F918F919C
:100140000F900FBE0F901F901895FC018585968526
:10015000029751F48281882321F085B3856085BBA5
:10016000089585B38A7F85BB0895809107018095A6
:10017000809307010895EF92FF920F931F93F894D5
:100180000E948B020E94670082E08093EE0160E093
:1001900070E080E090E00E949D02789484B38560D6
:1001A00084BBAA9A82E3E82EF12C00ED17E021E04F
:1001B00030E040E050E060E070E085EB90E00E94CD
:1001C000E4000E94DC01FDCFCF92DF92EF92FF921C
:1001D0000F931F93CF93DF93EC016B01A0E0B0E08E
:1001E0009A2FFD0184E0EE0FFF1F8A95E1F7EA0FD9
:1001F000FB1FE85FFE4F8785882329F09F5F1196DC
:10020000AC30B10569F7692F70E0FB01A4E0EE0F97
:10021000FF1FAA95E1F7E60FF71FE85FFE4FD183B6
:10022000C083D382C2825583448337832683E114FB
:10023000F10411F4108A08C082E3E816F10411F405
:1002400081E001C082E0808BFB0134E0EE0FFF1FF4
:100250003A95E1F7E60FF71FE85FFE4FA089B0E09F
:10026000AC52BE4F8C91982F9E0D96878F5F8C93CA
:100270001187008781E08787F894209101013091F0
:1002800002014091030150910401C801A0E0B0E0D7
:10029000820F931FA41FB51FFB0124E0EE0FFF1F69
:1002A0002A95E1F7E60FF71FE85FFE4F82879387F5
:1002B000A487B5877894DF91CF911F910F91FF901C
:1002C000EF90DF90CF900895CF92DF92EF92FF9260
:1002D0000F931F93CF93DF93DC01EB01690120E0C3
:1002E00030E0622FF90174E0EE0FFF1F7A95E1F71D
:1002F000E20FF31FE85FFE4F8785882331F06F5FC1
:100300002F5F3F4F2C30310561F7262F30E0F90188
:1003100064E0EE0FFF1F6A95E1F7E20FF31FE85F5D
:10032000FE4FB183A083D383C28355834483D78296
:10033000C682E114F10411F4108A08C082E3E816C1
:10034000F10411F481E001C082E0808BB90194E0F6
:10035000660F771F9A95E1F7620F731F685F7E4FF4
:10036000EB01E889F0E0EC52FE4F8081982F9E0D62
:100370009E878F5F80831987088781E08F87209110
:100380000101309102014091030150910401C80123
:10039000A0E0B0E0820F931FA41FB51FFB0182876E
:1003A0009387A487B587DF91CF911F910F91FF901D
:1003B000EF90DF90CF900895EF92FF920F931F93ED
:1003C000CF93DF93F894E0900101F0900201009147
:1003D00003011091040178941092D7018091DA0101
:1003E0008F5F8093DA018091DA01883C49F4809133
:1003F000D90186958093D8011092D9011092DA0123
:100400004FEF5FEF20E030E0F901A4E0EE0FFF1FB7
:10041000AA95E1F7E20FF31FE85FFE4F8785882377
:1004200099F08091D7018F5F8093D7018285938562
:10043000A485B585E816F9060A071B0728F0868506
:10044000851710F45685422F2F5F3F4F2C30310512
:10045000D9F64F3FB9F18091D9018F5F8093D901CF
:10046000842F992787FD9095EC01E4E0CC0FDD1FE8
:10047000EA95E1F7C80FD91FC85FDE4FE881F9811F
:100480006C817D818A819B8109958E819F81892BD9
:1004900049F41F86E889F0E0EC52FE4F80818150DC
:1004A000808310C02A853B854C855D85888599852C
:1004B000A0E0B0E0820F931FA41FB51F8A879B871F
:1004C000AC87BD8781E0DF91CF911F910F91FF90A5
:1004D000EF900895AC0120E030E0F901B4E0EE0FB8
:1004E000FF1FBA95E1F7E20FF31FE85FFE4F80812F
:1004F00091818417950749F41786E089F0E0EC5262
:10050000FE4F80818150808308952F5F3F4F2C30B4
:10051000310519F7089580E090E0FC0124E0EE0F2A
:10052000FF1F2A95E1F7E80FF91FE85FFE4F1786D6
:1005300001968C30910589F708958091EE01880F1E
:1005400081608093720080E280937000E1E7F0E0C8
:1005500080818C7F808385EC8093740081E090E0C3
:100560009093DD018093DC011092DB018FEF80938B
:10057000ED011092EC011092EB010895582F80913B
:10058000DC019091DD01019759F18091DC0190919E
:10059000DD01049771F524C08C91F901E252FE4F00
:1005A00082838091EA019D9189278093EA012F5FE0
:1005B0003F4F2617370784F31092DB014093DF018A
:1005C000852F90E0880F991F8093DE0185EA809344
:1005D000740082E090E09093DD018093DC01089547
:1005E0008FEF8093EA01DB0120E030E0642F70E0C0
:1005F000E0CF08951F920F920FB60F920BB60F9295
:100600001124EF92FF920F931F932F933F934F93D9
:100610005F936F937F938F939F93AF93BF93EF936A
:10062000FF938091DC019091DD01817C09F48DC004
:100630008091710090E0887F907080389105A1F0E2
:10064000813891054CF48036910509F46AC08037F1
:10065000910509F078C065C08039910529F0803A8C
:10066000910509F070C06DC08091DC019091DD01B1
:100670008034910551F4809173008093DF018FEFF6
:100680008093ED0180E890E047C08091DC0190917B
:10069000DD018038910509F054C09091DB01809113
:1006A000DF019817A0F48091DB01E82FF0E0909132
:1006B0007300E252FE4F92838F5F8093DB01909133
:1006C000ED018091730089278093ED013AC08091FC
:1006D00073008093EA019091ED018091EA019817EF
:1006E00019F081E090E002C082E090E09093EC018C
:1006F0008093EB01EE24FF2400E010E020E030E0E6
:1007000040E050E06EED71E085EA90E00E94640107
:100710001092DB0181E090E09093DD018093DC0199
:1007200010C0809173008093DE011092EC01109252
:10073000EB011092DB0185EC8093740080E490E083
:100740006AC085EC74C085E472C080917100282F66
:1007500030E0287F30702831310599F0283231059A
:10076000B9F02830310509F05BC08091DE0180933B
:10077000730085E8809374003093DD012093DC01E1
:1007800058C01092DB018091DF01809373003EC05E
:100790009091DB018091DF01981751F48091EA017B
:1007A000809373008091DB018F5F8093DB012EC00B
:1007B0002091DB018091DF0130E090E00196281765
:1007C0003907C1F485E98093740080E290E090934A
:1007D000DD018093DC01EE24FF2400E010E020E046
:1007E00030E040E050E060E070E08DE992E00E948F
:1007F00064011FC09091DB01E92FF0E0E252FE4F4F
:100800008281809373009F5F9093DB0185E88093E2
:10081000740080E190E09093DD018093DC0109C0D9
:1008200084E090E09093DD018093DC0185E080938B
:100830007400FF91EF91BF91AF919F918F917F9144
:100840006F915F914F913F912F911F910F91FF9069
:10085000EF900F900BBE0F900FBE0F901F9018954A
:04086000F894FFCF3A
:00000001FF
